:020000020000FC
:1000000058CD0000000000001FC0A4C18DC000003A
:10001000000097C00000000000000000020304067A
:10002000080C10182030406080000406080C1018DE
:100030002030406080A0C0000003070F1F000505AE
:100040000D050305030302004FB662FD0CC05520E9
:1000500041F00994C52DC095089483FDC795C4BD92
:1000600064604FBE1895C0916400089483FDC795E5
:10007000C4BD6B7FC0916400CF3F09F41EC070FF08
:100080001AC082FD05C04FBEC198979895981895E3
:1000900076FD0EC065FD0CC0C091B100C0FD929808
:1000A000C1FD9398C2FD9498CAEFC095CA95F1F727
:1000B000C198979895984FBE189524BCCC27C064DA
:1000C000C8BF6460F8CFC6CF70FFC4CF65FDC2CF94
:1000D000C19AC0CF70FFBECF65FDBCCF979ABACF93
:1000E00070FFB8CF65FDB6CF959AB4CF929A70FFE6
:1000F000B1CF65FDAFCFC7E0CA95F1F7C19AAACFDE
:10010000939A70FFA7CF65FDA5CFC7E0CA95F1F719
:10011000979AA0CF949A70FF9DCF65FD9BCFC7E0C3
:10012000CA95F1F7959A96CF4FB6C9B7CF7EC9BF9A
:100130006E7FCCB5CE0DDDB5DF1DDBBDCABD4FBEBC
:1001400018953FB68F7EA9B7A072A2118061A9B79A
:10015000AF7DA9BFA9B7AE7FA9BF7894A091680071
:10016000AA2341F085FD2BC0A0916800AA95A09319
:10017000680025C040E050E085FD15C0A6B396FD9F
:10018000A095A0FD4FEFAEB5A06496FDAF7BAEBDD0
:10019000AA27A062A8BF8D7FA6B396FDA095A0FD5B
:1001A0005FEF451739F7A8E161FDA093680085FD71
:1001B00003C0A8E1A093680040939600816085FD8C
:1001C0000EC0A0916900AA2331F0A0916900AA9500
:1001D000A093690004C08061AA27A062A8BF80FF25
:1001E0003DC0A09196004A2F61FF8E7F85FD18C00B
:1001F000403F08F040EFA42FA295AF704A0F5091F6
:10020000B600533069F0A695A69550FD01C0A6959D
:1002100052FD03C0A41B4A2F03C04A0F08F44FEF3E
:10022000A0919F004A1708F44A2F40936100A72F1E
:10023000A670A1F073FD12C0A0917000AA0FAA0FC2
:1002400050919E0056955695541708F0452F4A0F29
:100250004093610018F4AFEFA0936100A09161009A
:10026000A093630040916300A0919B004A1708F09F
:100270004A2F542EA091A000AA2309F422C0542F83
:100280005A1B10F4A42F50E0BA2E8894AA1FAA2E4D
:10029000A091A200A095AA22A50E58F0A091A100BD
:1002A000A21509F0AA95AA0EA093A10048F04A2D24
:1002B00008C0A091A100BA1608F0A395A093A100D0
:1002C0004FEF409364007F7B485F08F07064A52D7A
:1002D000A03408F06860A0916000A395A09360002E
:1002E00059F0F894A9B7A160A9BF84FF03C0A9B7CA
:1002F000A062A9BF3FBE1895A0917400A395A093DA
:10030000740041E050916800552329F085FF03C037
:100310005A9550936800A0919600A13018F0209251
:1003200099000DC020929A002092A300A0919900FC
:10033000AF5FA093990018F0AFEFA0939900F894E5
:10034000A9B7A160A9BF84FF03C0A9B7A062A9BFD4
:100350003FBE18953FB646B557B58F7EA9B7A07278
:10036000A2118061A9B7AF7DA9BFA9B7AE7FA9BF10
:10037000789481FD25C0AEB5AF7B96FDA064AEBD7F
:100380008260A6B396FDA095A0FF05C040936500CE
:100390005093660041C1AEB5A06496FDAF7BAEBD83
:1003A000AA27A062A8BF8D7F85FF01C028C140E0B9
:1003B000A6B396FDA095A0FD22C14093960011C161
:1003C000AEB5A06496FDAF7BAEBD8D7F61FF72C000
:1003D000AEB5AF7B96FDA064AEBDAA27A062A8BF54
:1003E00082604093910050939200A0908F004A1930
:1003F000B09090005B09BB24A22C4C38520518F435
:100400002092950049C0A091D400AA2359F1483CFC
:10041000520528F4A0E1BA2EAAE0AA2E23C048363D
:10042000A1E05A0728F4A8E0BA2EAFE0AA2E1AC01D
:10043000403DA2E05A0728F4A4E0BA2EAEE1AA2E6D
:1004400011C0403AA5E05A0728F4A2E0BA2EACE366
:10045000AA2E08C04839A8E05A0720F4A1E0BA2E15
:10046000A8E7AA2EC42EA0919300CA1AD52EA09157
:100470009400DA0ADD202AF4AFEFC094D094CA1AAF
:10048000DA0A20929500A8E0A210A0E0CA14DA06C9
:1004900018F4A1E0A093950040939300509394002A
:1004A000409191005091920040938F0050939000A2
:1004B00042E097C0A09165004A1BA09166005A0BCC
:1004C00094FD82C093FD80C092FD7CC086FF03C076
:1004D000D52EC42E0CC05695479591FD73C05695E8
:1004E000479590FD6FC0D52EC42ED694C79461FD5C
:1004F00019C0AC2DAC51AD2DA24008F005C0DD20D7
:1005000089F4AC2DA85C70F4A0916700A395AA2390
:1005100011F0A0936700AA3008F471C020929600F1
:1005200081606DC0A0916700AA2319F0AA95A093DD
:100530006700A22C5091BA0097FD06C0A090C80099
:10054000533011F4A090D000AAEFAA0EA22DA21D44
:10055000CA18DA0A4FB74170533049F4442321F0E6
:1005600087FD05C0806803C087FF01C08F774423E3
:1005700059F0533031F4AFEFC094D094CA1ADA0A6C
:1005800003C040E050E020C0533049F4CC0CDD1CE7
:10059000AAE0CA1AD20818F4A0E0CA2ED22CAFEFF3
:1005A000CA16D20418F04FEF50E00EC0A091AC0074
:1005B000CA9E412D000C441F50E008F012C04FEFBE
:1005C00050E00FC05695479594FF07C0552309F09A
:1005D0004FEFA42FA6954A0F521D4F3F520508F02A
:1005E0004FEF40939600816061FF09C0AFE1A09595
:1005F000A923AB299A2F8F7DBB2009F48062A8E143
:10060000A093680085FF03C0AAE0A093680061FD85
:1006100003C085FD01C08F7E85FD03C0A6E0A093C9
:100620006900F894A9B7A160A9BF84FF03C0A9B766
:10063000A062A9BF3FBE189511E00AC013E008C030
:100640001AE006C01EE104C014E602C018EC00C0A7
:1006500005E1BB27BA95F1F70A95D9F71A95C1F7C5
:1006600008952AE338E709C020E33CE806C02AE2FF
:1006700034EB03C025E238EC00C012E0BB27939AAC
:10068000BA95F1F7979ABA95F1F79798BA95F1F765
:100690009398BA95F1F7123009F0C19A123009F423
:1006A000959AB091AD00BA95F1F7123009F0C19862
:1006B000123009F49598B7E8BA95F1F71A95F1F662
:1006C000022FB22FBA95F1F70A95D9F73A95A9F604
:1006D000939A0895221B39E0001F3A9509F4089572
:1006E000221F211B18F4210F8894F6CF0894F4CF11
:1006F000622C722CB0E08894B395221F331FE0F770
:10070000379527958894912E802E020B130B10F4A9
:10071000192D082D10F4889401C00894661C771CCC
:10072000BA9571F7172D062D0895322D11232AF44D
:100730003A9500951095031B130BF894029F712CAA
:10074000002D129F912C802C7894780C172D921CE0
:10075000292DB4E06B2E2695179507956A94D9F745
:10076000332321F000951095031B130B0895089572
:1007700010917B00169500917A000795B0917E004C
:10078000B01B0B2FB0917F00B10B1B2F28F400384A
:10079000BFEF1B0740F009C00F37120508F405C072
:1007A0000FE710E002C000E81FEF009383001093F2
:1007B0008400089500918300B09180000B0F109188
:1007C0008400B09181001B1F20E03091840033230E
:1007D0000AF42A95B09182002B1F1AF4203F40F0B2
:1007E0000AC02F3008F407C00FEF1FEF2FE003C03F
:1007F00000E010E020EF30916300B0919B003B17C8
:1008000018F4323030F009C0B0918400BB235AF0A4
:1008100004C0B0918400BB2332F400938000109395
:1008200081002093820008952091D70000918300D9
:10083000000F10918400111F78DF11232AF4003873
:10084000BFEF1B0740F009C00F37120508F405C0C1
:100850000FE710E002C000E81FEF002352F0B09154
:100860006200B01B0B2F18F0013008F00AC001E045
:1008700008C000950F5FB09162000B0F08F001C037
:100880000FEF0093850008952091D800009181001A
:10089000109182004ADF11232AF40130BFEF1B07B9
:1008A00040F009C00F3F120508F405C00FEF10E03B
:1008B00002C001E01FEF112352F0B0918500B01B80
:1008C0000B2F18F0013008F00AC001E008C00095B5
:1008D0000F5FB09185000B0F08F001C00FEF009380
:1008E000630008950FEF677F71FD29C072FD09C095
:1008F0006860B0917B00BA3020F0B52DB03408F4B8
:10090000677FB091D300BB23D1F0B0917B00BB23B4
:10091000B1F00FEF10917B00DDDEF894B091730021
:1009200072FDB5E00B9F112D002D7894112309F075
:100930000FEFB0919E000B1710F400919E000093F2
:100940009D00089500917A0010917B0000541140A1
:10095000B0919D0010F4BA9501C0B39511F0B09319
:100960009D00089500C008952091B500B6B1B6FD70
:10097000FBCF04B115B1B6B1BF77B6B9B091AA003B
:10098000B395B093AA00B83060F12092AA00B0915C
:10099000D200BB2321F1112329F0B091AB00BF3F5E
:1009A00061F009C0B091AB000B1739F020F4BB2304
:1009B00021F0BA9502C0B395E1F300919B00B0938A
:1009C000AB00BA3F50F400ECB93F38F400E8B83F50
:1009D00020F400E4B73F08F400E000939B007F7E22
:1009E0000895B0919B00B39511F0B0939B00B09126
:1009F000AA00B73009F47061089502E3F894B09149
:100A0000D9000B9F012D000C001F7894B0919B0022
:100A10000B1710F000919B0000936100009363009E
:100A2000502E0093640000939E00089520927A0057
:100A3000B0EFB0937B000895F8940CB51DB52091EC
:100A40007400789430917500609076000093750082
:100A500010937600031B160971FD03C077FD7DC05E
:100A600027C070907700209377002709222311F088
:100A70000FEF1FEF8090780090907900309378000E
:100A8000609279000091750010917600081919099B
:100A900020917A0030917B0036952795020F131F25
:100AA00010F40FEF1FEF00937A0010937B0029C022
:100AB00020917A0030917B003901B4E08B2EB2E0B6
:100AC0009B2E343010F08A949A94383010F08A9427
:100AD0009A94769467948A94E1F7261937099920B5
:100AE00021F0169507959A94E1F7200F311F209376
:100AF0007A0030937B0028F43FEF30937A003093F4
:100B00007B00323008F4706871FF02C0B3E00DC0A2
:100B1000B091C40000917100023838F0B395003AEA
:100B200008F0B395B63008F0B5E09B2EB4E08B2EFC
:100B300010917B0000917A0024E0169507952A9584
:100B4000E1F70819120928F0B02FB250B12FB209FD
:100B500010F402E010E0980126C020917A00309154
:100B60007B0039017694679466946694669426199E
:100B7000320906950695200F321D20937A00309396
:100B80007B00323008F07F7704E036952795369564
:100B9000279526952695201B10F0223008F422E098
:100BA00089019090C40060FDFECFE0908B00F09032
:100BB0008C006160B9B7B061B9BF380177FD41C041
:100BC0007694679400938B0010938C00B92DB3300A
:100BD000E1F0B0FD04C0060D171D930106C0000F23
:100BE000111F0250120922E030E0B92DB33068F035
:100BF00020938D0030938E0000938700109388001F
:100C00006092890070928A003AC000938D00109320
:100C10008E00209387003093880060928900709244
:100C20008A0071FF0DC0BFE0B0938D0020928E004E
:100C3000B093890020928A00B0938B0020928C00A0
:100C40001EC0669400938B00B92DB33091F0B0FDB7
:100C500003C0060D262D03C0000F025022E0B92D5F
:100C6000B33038F020938D000093870060928900A4
:100C700006C000938D002093870060928900009148
:100C80007C0002FD0350013029F495FD0AC0B0E05C
:100C9000B7B909C0023019F4B7E0B7B904C095FD7F
:100CA000F6CFB6E0B7B90091A200000F10F4BBE692
:100CB0000B270093A20060FDFECFB2E0B0936E0060
:100CC0006160B9B7B061B9BFB72FB670D1F02091EC
:100CD0007A0030917B00369527953695279571FFE0
:100CE00002C0B0E43B0FF8940CB51DB5020F131F02
:100CF0001BBD0ABD6160B0E1B8BFB9B7B061B9BF93
:100D000078940895606120927D0020E067FD20E2E4
:100D100006C0606120927D0020E267FD20E001E0D6
:100D200011E077FD11C0B72FB67009F06F7E14E1A6
:100D300000917B00069509F403950F3008F00FE051
:100D400071FF02C004E114E160FD0FC0B0917D00AD
:100D5000BB2359F071FF06C0B0916E00BA95B093F5
:100D60006E0011F4706247C0ABDFB0B7B77FB0BFA1
:100D7000B8B1B0B7B860B0BFB0917D00B395B093D3
:100D80007D00B8B177FD06C0B1E071FDB3E0BA9562
:100D9000F1F7B8B1B072B21709F022C071FF05C007
:100DA0000395011708F00A95CFCF64FD05C00395A0
:100DB000011708F0B4CFC8CF6F7EF8943CB56DB47E
:100DC00070907A0080907B00370D681C6BBC3ABD38
:100DD0006160B0E1B8BFB9B7B061B9BF78949FCFD7
:100DE000B0916D00B13008F49ACF64FD98CF0A95A8
:100DF00009F0AACF7F7D20918D0030918E00F8946C
:100E0000B0E1B8BF0CB51DB5020F131F1BBD0ABD65
:100E1000E0908700F09088006160B9B7B061B9BF19
:100E20007894B72FB67039F0B0916D0072FFB3951A
:100E3000B0936D0009C075FF07C067FD05C064FD74
:100E400003C0BF91BF91EDC4089500E063FF03C0EC
:100E500064FF01C001E0F89410917100B7E01B9F9E
:100E6000212D102D7894200F2695179526951795EE
:100E70002695179510937100183718F4B8E7B093BA
:100E8000710000917100B09172000B1720F0606248
:100E9000C1989798959860FDFECFE0908900F090FA
:100EA0008A006160B9B7B061B9BF0895B2E095FD3D
:100EB0000AC0F894B0937C00939A929862FF01C0A4
:100EC000959A7894F4C0F894B0937C00939A94988F
:100ED00062FF01C0C19A7894EAC0B3E082FF24C0E7
:100EE00095FD11C002E0F894B0937C00E0E8F0E0DA
:100EF0000093B1009598949A62FF02C0979A01C03E
:100F000093987894D4C002E0F894B0937C00E0E821
:100F1000F0E00093B100C198929A62FF02C0979AE4
:100F200001C093987894C3C095FD0BC0F894B0931A
:100F30007C00EAE6F0E0959862FF01C0979A789409
:100F4000B6C0F894B0937C00EAE6F0E0C19862FF86
:100F500001C0979A7894ABC0B4E095FD0AC0F894AC
:100F6000B0937C00929A949862FF01C0979A78940B
:100F70009EC0F894B0937C00949A929862FF01C04E
:100F8000979A789494C0B5E082FF24C095FD11C073
:100F900001E0F894B0937C00E6E7F0E00093B10044
:100FA0009798939A62FF02C0C19A01C09298789470
:100FB0007EC004E0F894B0937C00EAE8F0E000938F
:100FC000B1009798939A62FF02C0959A01C09498D5
:100FD00078946DC095FD0BC0F894B0937C00E4E666
:100FE000F0E0979862FF01C0C19A789460C0F894CD
:100FF000B0937C00E0E7F0E0979862FF01C0959A1B
:10100000789455C0B6E095FD0AC0F894B0937C0082
:10101000949A939862FF01C0C19A789448C0F8945A
:10102000B0937C00929A939862FF01C0959A78944D
:101030003EC0B1E082FF24C095FD11C004E0F894E9
:10104000B0937C00EAE8F0E00093B100C198929A76
:1010500062FF02C0959A01C09498789428C001E07C
:10106000F894B0937C00E6E7F0E00093B100959827
:10107000949A62FF02C0C19A01C09298789417C0F6
:1010800095FD0BC0F894B0937C00E0E7F0E0C198C8
:1010900062FF01C0959A78940AC0F894B0937C00DE
:1010A000E4E6F0E0959862FF01C0C19A78946F7D04
:1010B000089523E630E0F9012092B100C198979895
:1010C0009598929A939A949A6B7F0895A2EBB0E0C8
:1010D0000FEF0D930D930D930D9303E00D9304E02B
:1010E0000D930AE00D9303E00D9301E00D9301E0F1
:1010F0000D93AEEBB0E001E00D930FEF0D930D9368
:101100000D930D930D9303E00D930FEF0D930FEFE0
:101110000D930D9305E20D9300ED0D930AEF0D93E2
:101120000AEF0D9304E00D930FEF0D9301E00D9383
:1011300000E00D930AE70D930FEF0D9300E00D9380
:1011400001E00D9300E00D9303E00D9300E00D939B
:1011500008952091B9008B7F233009F48460B09109
:10116000BA00B33019F09F7DB1FD90629F7BB091C2
:10117000BB00B1FD9064223011F0886001C0877F10
:1011800008950A95E00FF21DB4910895ECE1F0E0A6
:101190000091B200F6DFB093D700ECE1F0E00091EF
:1011A000B300EFDFB093D800EAE2F0E00091B800BE
:1011B000E8DFB093D9000091B800023008F402E0F3
:1011C00000937300B091CE000FEFB23009F400EA43
:1011D000B33009F402E800937200E8E3F0E0009114
:1011E000D500CFDFB093A000089508952091C800E6
:1011F0003091C900B091BA00B33009F43E5097FF66
:1012000002C020E03FEFB32FB21B6B2EB25810F498
:10121000B2E86B2E00E00395609EB12DBD57D8F368
:101220000093AC0008959068E1DF0CDA20E030E034
:10123000B0E16B2E03DAB09196002B0F321D6A9449
:10124000C9F7B4E036952795BA95E1F7822E9F77D6
:10125000CDDF0895F894E3E0F0E0B9E0B7BFB491D2
:10126000B078C1F3F894A895B1B5B861B1BDB0E05C
:10127000B1BDB4E0BEBFBFE5BDBF1BDFB0E0B8BBD2
:10128000B2E1B7BBB0E0B5BBB0E0B4BBBCE1B2BB50
:10129000BCEBB1BB2224A0E0B0E02D92AA31E9F76B
:1012A000A0E6B0E00FEF2D920A95E9F7B1E0B09318
:1012B000A2000CDFEED2B6B1B460B6B90091CA009C
:1012C0000093AD00B1E0B0936A00F894BFD9C9D9DA
:1012D000B9D9CAD9B7D9CBD9B5D962D3B7D9B6D9C3
:1012E000B3D9F8940AEF1AEFA6B396FDA095A0FF24
:1012F0001FC01A95C9F70A95B1F7E0E0FCE1B59176
:10130000B43E39F4B591B03E21F4B591BF3F09F434
:101310000CC0E0E0F395F395B591B83F49F4B59171
:10132000B43931F4B591BA3A19F4EE27F695099427
:1013300010DF2CDF5ADF5ADF0091CA000093AD00A6
:10134000B8DEB2E0B3BFB2E0BEBDB2E0B5BDB1E55C
:10135000B8BFB9BFB0B7B77FB0BFB8B1B0B7B860AA
:10136000B0BF6AD97894FEDA20927000BEB5B0643E
:1013700096FDBF7BBEBDB9B7B062B9BFBB27B06237
:10138000B8BF8D7F63D9626033E02CE0B0919500E7
:10139000BB2321F42CE03A9509F4A3CF53D980FF65
:1013A000A0CF8E7FB0919600B23078F3B92FBF7185
:1013B0000091980000939700B0939800B01729F718
:1013C0002A9521F76D7FBEB5B06496FDBF7BBEBD8B
:1013D000BB27B062B8BF8D7FB091D400BB2321F48E
:1013E0008062B92FB0709B2F8F7B209267002CD921
:1013F00085FF05C0B0916700BA3008F080641ED93F
:1014000002E085FF01C000E0B0919600B017B8F38C
:10141000F89427D926D925D9789418D9209286000E
:10142000B091BA00B33009F474C008D9B091BE00CD
:10143000B13008F46EC0B0916A00B13008F469C0F0
:1014400085FD18C0B0919600BF3F08F462C0F894C3
:1014500011D97894F9D8B0919600B130C0F7F894CA
:1014600000D9EED8FED87894EFD8B0919600BF3F5F
:10147000B0F3C8C2B8E09B2E9068F894B7DE7894B9
:10148000E3D8F8949F77B2DE80909600B0919600F2
:10149000BF37789408F445C0CFD8F894EBD8789447
:1014A0009A9451F7C0DEB82DB550B093C900CED88C
:1014B000F8941CD27AD27894BAE09B2E9068F89473
:1014C00095DE7894C1D8F8949F7790DE809096004E
:1014D000B0919600BF37789478F7AED8F894C1D819
:1014E000AFD8BFD878949A9449F79DDEB82DBB5FEA
:1014F000B093C800ABD8F894F9D166D27894A4D848
:10150000F89474DE7894B0919600BF3F08F498CFB9
:1015100079C200919600B09186000B1710F00093ED
:10152000860092D801E0B091BA00B35009F405E00A
:10153000B0919600B01708F073CFF8949BD89AD862
:1015400099D8789483D820926A0020926B002092D8
:101550006C00B0916B00B395B0936B00BF3F71F519
:10156000B0916C00B395B0936C00B091CC0009E1E0
:10157000BA9559F002E3BA9541F00DE7BA9529F012
:101580000AEFBA9511F020926C00B0916C00B01780
:10159000A8F08FDD51D8B0916C00BA95B0936C0073
:1015A00020926B00B091CB00B093AD00F89462D85C
:1015B0007894B091CA00B093AD0046D841D8B091AC
:1015C0006800BB2319F485FF01C08BCE01E085FDC7
:1015D00001C006E0B0919600B01708F4BACFB09100
:1015E000BA00B35009F030D8B0916800BB2309F4B9
:1015F00078CEF8945EDD2092610020926200209205
:101600006300522C209264002092A1007894B09143
:10161000B700BB0FB0939F0020927E0020927F0006
:101620002092800020928100209282002092AA00C5
:1016300060E070E020927100B8E0B093AA007061A1
:10164000FBD7B2E074FDB1E0B7B9B6B1B068B06431
:10165000B6B9B6B1B6FDFDCF04B115B1B6B1BF771D
:10166000B6B9112309F00FEF0093AB007DD9B8E0B4
:10167000B093AA0070616DDDF894BFEFB0939B004A
:10168000BCD9B0916100B0939B00B0939C00B09323
:101690009D007894B1E0B0936100B09363005B2E3D
:1016A000B0936400B093A400B0919A00B093A300EB
:1016B000B091BA00B33019F49F7D87FD90627160DC
:1016C000726020926D009EDCB4DCB0D9B5D9AED981
:1016D000B3D9ACD91EDB4BD8B8DBE8DBADD912DB14
:1016E00066FD46D877FFFED877FD2CD9AEDBF5DB5B
:1016F000A3D90FDB66FD5ED8A8DB2EDC9DD902DB0B
:1017000066FD92D8A2DB3FDC97D903DB66FDBCD82F
:101710009CDB78DC91D9F6DAB2E074FDB1E0B7B9C0
:10172000B6B1B068B064B6B990DB83DC85D91CD99A
:1017300071FF21C0B0919E00B0939B00B0939C00BC
:10174000B0919A00B093A300B1E0B093A40018E167
:101750002CE0B0916D00B11740F07D7F7460209354
:101760006F00BFEFB0939B0006C0B0919600B13000
:1017700008F0B0CF60C072FF11C067FD0FC0B0911C
:101780006F00BA9519F47B7F7860A4CFB0936F0097
:10179000B0919600B13008F09DCF4DC020927000FE
:1017A000B091990002E81091D600112309F003E0EE
:1017B000B01708F040C085FF04C0B0916800BB239B
:1017C000D1F1B091BA00B33081F495FD03C087FD2B
:1017D00004C00BC087FF01C008C067FD06C0606879
:1017E000B0919E00B0939B008ACF00EF67FF05C0C9
:1017F000B0919E00B0939B0000E2B0917B00B017C7
:1018000008F468CF67FF17C06F779F7D87FD9062F0
:101810007460B2E1B0936F00B0919E00B0939B00F2
:1018200059CFB0917000B395B0937000B09196000D
:10183000BB2309F002C020927000F8943ADC80903B
:10184000B900B2E0B093B90084DC8092B900209274
:1018500061002092620020926300522C209264006A
:1018600020929F0060E070E07894EED622DC009138
:10187000D600002319F0C19A979A959AB6B1B46030
:10188000B6B985FF05C0B0917000B43008F029CD1D
:101890005CCEEDE0F0E023D00A3509F01BC0EEE0AD
:1018A000F0E01DD0053A09F015C03AE0A2EBB0E037
:1018B000E3E0F0E014D00D9331963A95D9F739E191
:1018C000AEEBB0E0EFE0F0E00AD00D9331963A9540
:1018D000D9F702C0FBDB0AD0E8E2F0E00895E19915
:1018E000FECFEEBBFFBBE09A0DB308951ED03AE0E9
:1018F000A2EBB0E0E3E0F0E00D910FD031963A9525
:10190000D9F739E1AEEBB0E0EFE0F0E00D9105D0B2
:1019100031963A95D9F712D00895E199FECF0DBBD3
:10192000EEBBFFBBE29AE19A0895EDE0F0E00FEF25
:10193000F4DFEEE0F0E00FEFF0DF0895EDE0F0E02F
:101940000AE5EBDFEEE0F0E005EAE7DF089530912D
:10195000AE000091AF00313011F40093B600323088
:1019600011F40093B700333011F40093B800343011
:1019700011F40093C400353011F40093B9003630EF
:1019800011F40093D500373011F40093CE003830B5
:1019900011F40093BA00393011F40093BB0008959C
:1019A00025E054D62A95E9F708955BD65DD65FD633
:1019B00061D646D656D658D65AD65CD641D651D6DA
:1019C00053D655D657D6089555D651D64DD649D665
:1019D00037D650D64CD648D644D632D64BD647D634
:1019E00043D63FD608958090AE009090AF0039D690
:1019F00038D637D625D68A94D1F73CD621D69A94B4
:101A0000E1F70895F894D1DF7894CADFC9DFB1E037
:101A1000B093AE00B1E0B093AF002092B000F89464
:101A2000E2DF7894B5E06B2E709096000FD6B091FF
:101A300096007B16C9F7B13018F0BF3F40F107C0E0
:101A400086DFF89453DFB1DFB8E0B1BDA9DF6A9457
:101A500059F7B091B000B395B093B000B33008F42B
:101A6000DECF9EDFB091AF00B395B093AF00F89496
:101A7000B091AE00BA95EEE3F0E0EB0FF21D0491E9
:101A800078940395B091AF00B01708F4C6CF88DF03
:101A900087DFB091AE00B395B093AE00B091AE00C9
:101AA000BA3008F4B7CF12DBF89420DFB8E0B1BD4C
:041AB00077DFD0CB41
:00000001FF
